:100000000C940D030C9454030C9454030C9454035B
:100010000C9454030C9454030C9454030C94540304
:100020000C9454030C9454030C946B0C0C943D0DE1
:100030000C9454030C9454030C9454030C945403E4
:100040000C9454030C94B1210C9454030C94540359
:100050000C9454030C94431B0C9454030C945403BD
:100060000C9454030C9454030C9454030C945403B4
:100070000C9454030C9454030C9454030C945403A4
:100080000C9454030C9454030C9454030C94540394
:100090000C9454030C9454030C9454030C94540384
:1000A0000C9454030C9454030C945403AA0DCC0DDB
:1000B000BF0ECC0DBF0E110E340EBF0E890E9C0E5E
:1000C00086118611B511B511F81132123F143F1483
:1000D0004B123F144013401313143F143F142A14BF
:1000E0000000F0A201002B002A00E10001540000F2
:1000F0001E00140004001D71010003521F001A00AD
:1001000015001B0001002800200009001600060051
:1001100052002C00210013001700190002522C0A73
:1001200022000A00070005000000E3005000010063
:1001300000000100000065004F00010000002B08D6
:100140000000297123000D000B000E000000E200EA
:1001500024000F001100100002522C0A2500180084
:100160000800360051002C0026001C000C0037004F
:10017000010028002700330012003871E600035206
:100180004C002B004C00E500E70000002A002B008B
:10019000E000E100010000001E00140004001D71D9
:1001A00034004D001F001A0016001B00E104E3009C
:1001B000200008000700060050002C002100150058
:1001C0000900190002524A00220017000A00050027
:1001D00000002B00500001000000E20000004C0075
:1001E0004F0001000000E6000000E20023001C00B8
:1001F0000B00110000002971240018000D001000F0
:1002000002524B0025000C000E0036005100280061
:10021000260012000F0037002F00E7002700130010
:100220003384387130004E004C003100E400E500AA
:10023000C1000000010001000100010001000000F8
:100240003A00010031020100010001003B001F02E1
:100250001E022202010001003C0025022E022302A0
:10026000010001003D002E002D00210201000100CF
:100270003E002D02340224020000010001000100B2
:100280000000010000000100010001000000010069
:10029000000001003F00350234023300000001007D
:1002A00040002F0226022F00010001004100300211
:1002B000270230000100010042002002340031001A
:1002C0000100010043003302350038000100010045
:1002D0004400450001000100010000000100010090
:1002E0000100010001000000010001000100010007
:1002F00001000100010001005000010001000100A7
:100300000100520051000100010001000100010044
:100310004F00010001000100010001000100010087
:1003200000000100010001000000010000000100C8
:100330000100010000000100000001000100210295
:100340002E002402000001000100240021001E00F4
:10035000360001000100250022001F0027000100D7
:1003600001002600230020003700010001002E02BA
:100370002D002502380001000100010001000100EC
:100380000100000001000100010001000100000067
:100390000100010001000100010001000100010055
:1003A000F2000100010001000100F000F100010075
:1003B000F400010001000100F3000100F50001005C
:1003C0000100010001000100000001000100010026
:1003D0000000010000000100010001000000010018
:1003E0000000010001000100010001000000010007
:1003F0000100010001000100A9000100010001004D
:100400000100AC00AA00B600010001000100AB0031
:10041000A80001000100010001000100010001002D
:1004200001000100AE0001000100000016034500BC
:10043000720067006F0044006F00780020004500E4
:100440005A00000016034500720067006F00440068
:100450006F007800200045005A00000004030904E2
:1004600009026D00040100A0FA0904000001030163
:100470000100092111010001223F00070581030845
:10048000000A090401000103010200092111010011
:1004900001224D000705820308000A090402000139
:1004A0000300000009211101000122360007058325
:1004B0000308000A090403000103000000092111D8
:1004C0000100012239000705840310000112011008
:1004D0000100000008EDFE07130100010200010504
:1004E000010906A101050719E029E7150025019575
:1004F0000875018102050819012905950575019105
:10050000029501750391010507190029771500254A
:1005100001957875018102C005010980A10185025C
:1005200016010026B7001A01002AB70075109501C0
:100530008100C0050C0901A1018503160100269C5C
:10054000021A01002A9C02751095018100C0050164
:100550000902A1010901A1000509190129051500D8
:10056000250195057501810295017503810105013C
:10057000093009311581257F9502750881060938F2
:100580001581257F950175088106050C0A3802152D
:1005900081257F950175088106C0C005010906A166
:1005A00001050719E029E715002501950875018166
:1005B0000295017508810105081901290595057540
:1005C0000191029501750391010507190029FF1595
:1005D0000025FF950675088100C00000000000009E
:1005E0000000000000010204060A0F17202C3A4AFE
:1005F0005D71879DB3C7DAE9F5FCFFFCF5E9DAC761
:10060000B39D87715D4A3A2C20170F0A0604020138
:100610000000000000000000000011241FBECFEF0A
:10062000DAE0DEBFCDBF04B603FE27C08091ED0146
:100630009091EE01A091EF01B091F0018730904BC5
:10064000A740B04BD1F41092ED011092EE01109240
:10065000EF011092F00114BE84B7877F84BF0FB6FC
:10066000F894A89580916000886180936000109252
:1006700060000FBEE0E0FFE3099511E0A0E0B1E00B
:10068000E4E0F7E402C005900D92A433B107D9F776
:1006900021E0A4E3B1E001C01D92AD3EB207E1F755
:1006A0000E94B2090C9480230C94000061110BC0CD
:1006B000FC018281882321F085EE0E94201003C076
:1006C00085EE0E94E81080E090E008950895609122
:1006D000B1017091B2018091B3019091B4010E9477
:1006E000701A56985E9825982D9826982E982798D7
:1006F0002F98813019F0823021F00895259A2D9A93
:100700000895269A2E9A08950C94670356985E9839
:1007100025982D9826982E9827982F988FEF90E05F
:10072000909389008093880090938B0080938A0037
:1007300090938D0080938C00259A2D9A2FEF80E75F
:1007400092E0215080409040E1F700C00000269ADE
:100750002E9A2FEF80E792E0215080409040E1F701
:1007600000C00000279A2F9A2FEF80E792E02150D7
:1007700080409040E1F700C0000025982D982FEFB1
:1007800080E792E0215080409040E1F700C00000F7
:1007900026982E982FEF80E792E0215080409040DD
:1007A000E1F700C0000027982F9856985E9825988A
:1007B0002D9826982E9827982F98089589EA809347
:1007C000800089E08093810024982C983F988AB11A
:1007D0008F748AB96E98479A8BB1806B8BB9769A71
:1007E0000E9486030C94660380E28093000180914E
:1007F000340181110EC00E94430481E080933401D2
:100800002FEF83ED90E3215080409040E1F700C04E
:10081000000080E40E9449048093000181112EC0F1
:100820000E94730480930001811128C00E94730408
:1008300080930001811122C08FE30E947304809392
:10084000000181111BC00E946B0480E40E944904D6
:1008500080930001811112C08CE00E947304809388
:10086000000181110BC00E9473048093000181116B
:1008700005C08FE30E947304809300010E946B0403
:100880008091000108951092B9008AE08093B80029
:10089000089594EA9093BC009091BC0097FFFCCF20
:1008A0009091B900987F983021F0903111F081E05B
:1008B00008958093BB0084E88093BC008091BC00C5
:1008C00087FFFCCF8091B900887F883111F0803498
:1008D00071F780E0089584E98093BC008091BC00AA
:1008E00084FDFCCF08958093BB0084E88093BC0016
:1008F0008091BC0087FFFCCF9091B900987F81E088
:10090000983209F480E0089584E88093BC008091D7
:10091000BC0087FFFCCF8091BB000895809100014F
:10092000811115C080E40E94490480930001811167
:100930000CC082E10E94730480930001811105C004
:100940008FEF0E947304809300010E946B0484B1B6
:10095000807F84B985B1807F85B98AB1837F8AB968
:100960008BB1837F8BB93E98469808950E94F4031B
:10097000809300010E948E0480B38C7080BB81B391
:10098000836F81BBE4E4F1E0A6E3B1E011921D9234
:1009900081E0E235F807D1F70C94DE039F92AF9225
:1009A000BF92CF92DF92EF92FF920F931F93CF935C
:1009B000DF9380910001882379F0809135018F5F6A
:1009C00080933501811108C00E94F40380930001D7
:1009D000811102C00E94860386E3E82E81E0F82E92
:1009E0008701C0E0D0E0BB24B39492E0A92ECC24D0
:1009F000C394D12CC730D10500F58091000181113D
:100A000064C080E40E94490480930001811112C0F7
:100A100082E10E9473048093000181110BC0C60122
:100A20000C2E01C0880F0A94EAF780950E94730487
:100A3000809300010E946B0448C0CA30A1F028F4E2
:100A4000C83059F0C93061F005C0CC3089F070F081
:100A5000CD3089F0209A289810C0219A29980DC08D
:100A6000229A2A980AC0239A2B9807C0529A01C04A
:100A7000539A5B9802C03E9A4698E0EAEA95F1F7ED
:100A80008FB181708B25799902C032E001C030E0CE
:100A9000832B7C9902C034E001C030E0832B7D9928
:100AA00002C028E001C020E0822B7E9902C090E1C4
:100AB00001C090E0892B9FB19095991F9927991FAC
:100AC0009295990F907E892B0FC080910001811122
:100AD0004AC080E40E94490480930001882381F188
:100AE000912C0E946B04892DD8019C91981719F0C4
:100AF0008C93A09201010E948E0421960F5F1F4FDC
:100B0000CE30D10509F076CF80910101882369F1BB
:100B1000815080930101882339F0EFE9FFE031979C
:100B2000F1F700C0000021C0E4E4F1E0D7018D91AD
:100B30007D018193B4E4EB16B1E0FB06B9F715C073
:100B400083E10E947304809300018111C9CF81E485
:100B50000E944904809300018111C2CF0E94840445
:100B6000982E9094BECF80E0BFCF0E94840381E096
:100B7000DF91CF911F910F91FF90EF90DF90CF9079
:100B8000BF90AF909F900895E82FF0E0EC5BFE4F90
:100B90008081089508958B3B910580F4883A9105F2
:100BA00048F5853A9105D8F48430910508F0B2C033
:100BB000019709F06EC081E090E00895803E9105B4
:100BC00008F467C0883E910508F4A4C09C01205F2A
:100BD00031092031310508F05CC090650895853AEF
:100BE000910509F459C0863A910509F058C082E888
:100BF00090E40895883A910509F454C0893A910522
:100C000009F453C08A3A910509F452C08B3A910510
:100C100009F451C08C3A910509F450C08D3A910500
:100C200009F44FC0803B910509F44EC08E3A9105FE
:100C300009F44DC08F3A910509F44CC0813B9105F0
:100C400009F44BC0823B910509F44AC0833B9105EE
:100C500009F449C0843B910509F448C0853B9105DE
:100C600009F447C0863B910509F446C0873B9105CE
:100C700009F445C0883B910509F444C0893B9105BE
:100C800009F443C08A3B910509F442C080E094E432
:100C9000089580E090E0089581E890E4089583E865
:100CA00090E4089582EE94E4089589EE94E4089522
:100CB0008AEE94E4089585EB94E4089586EB94E439
:100CC000089587EB94E408958CEC94E408958DECFA
:100CD00094E4089583E895E408958AE895E40895F6
:100CE00082E995E4089584E995E4089581E296E423
:100CF000089583E296E4089584E296E4089585E2F7
:100D000096E4089586E296E4089587E296E40895CD
:100D10008AE296E40895089524E5829FC001112493
:100D2000FC0126E0729FE00DF11D1124E60FF11D7C
:100D3000EE0FFF1FEC51FF4F859194910895880F9E
:100D4000991FFC01E05AF040859194910895880F15
:100D5000991FFC01E052FF4F85919491089524E57D
:100D6000829FC0011124FC0146E0749FE00DF11D3B
:100D70001124E60FF11DEE0FFF1FEC51FF4F85917F
:100D800094919C013A9521154FE1340708F425C14F
:100D90003F512115304120F49F700E94A70608950D
:100DA0009C0130532115304118F49927906C089517
:100DB000811520E5920769F40E9461144FEF84E3E6
:100DC0009CE0415080409040E1F700C000000C944E
:100DD000681B813020E5920731F48091CC0181605D
:100DE0008093CC0108959C0130552115304108F0C5
:100DF0005CC0292F33272F70332721303105E9F4C8
:100E0000AC0164E0440F551F6A95E1F74427537025
:100E1000BC016370772702C0220F331F6A95E2F787
:100E20003C68242B352B73E0880F991F7A95E1F7E6
:100E300080769927822B932B08952230310529F44F
:100E4000982F8827816F906A089523303105A1F487
:100E5000AC0133E0440F551F3A95E1F7407E5770DF
:100E60008370992721E030E002C0220F331F8A955A
:100E7000E2F7C9019C6816C02430310531F5AC0198
:100E800023E0440F551F2A95E1F7407E5770837089
:100E9000992721E030E002C0220F331F8A95E2F744
:100EA000C9019A68842B952B08959C013057211510
:100EB000304118F49F70906208959C0130582115BC
:100EC000304118F49F70906A0895803E9105E0F4D7
:100ED000803C910558F58133910509F46FC048F4C1
:100EE0008932910509F463C08A32910509F46DC015
:100EF00072C089339105E9F082389105D1F08533CC
:100F0000910509F44DC067C0833E910581F138F425
:100F1000803E9105B9F0823E9105D9F05CC0863ED5
:100F2000910561F1873E9105A1F155C00E949F0690
:100F300008952091DE0120FD02C021FF4CC080EE0B
:100F400090E049C08091DE0180FFF9CF89E390E015
:100F500042C08091DE0182FF0EC08091DE0184FFDD
:100F600003C080E090E037C083EE90E034C0809111
:100F7000DE0182FFF2CF82EE90E02DC08091DE0193
:100F800083FF0BC08091DE0184FDEBCF87EE90E004
:100F900022C08091DE0183FFF5CF86EE90E01BC07A
:100FA0008091DE0185FF07C089E290E014C0809146
:100FB000DE0185FFF9CF85E390E00DC08091DE0171
:100FC00086FF07C08AE290E006C08091DE0186FFBE
:100FD000F9CF81E390E00E94CB05089508958091B8
:100FE00062010895CF93DF9300D01F92CDB7DEB793
:100FF0009C018091E401843019F593E099833B834F
:101000002A839093E9008FEF9091E800815095FD3D
:1010100006C095ED9A95F1F700008111F5CF80910A
:10102000E80085FF0DC040E050E063E070E0CE01D5
:1010300001960E945F0A8091E8008E778093E80015
:101040000F900F900F90DF91CF910895CF93DF9382
:1010500000D01F92CDB7DEB72091E401243021F5F6
:1010600022E029839B838A8383E08093E9008FEFCA
:101070009091E800815095FD06C095ED9A95F1F7A5
:1010800000008111F5CF8091E80085FF0DC040E0A0
:1010900050E063E070E0CE0101960E945F0A80910B
:1010A000E8008E778093E8000F900F900F90DF910B
:1010B000CF9108959C018091E4018430F9F482E09D
:1010C0008093E9009FEF8091E800915085FD06C074
:1010D00085ED8A95F1F700009111F5CF8091E80038
:1010E00085FF0CC040E050E065E070E0C9010E945F
:1010F0005F0A8091E8008E778093E8000895CF938F
:10110000DF93EC018091E401843009F046C09091B6
:101110000C019923D9F090910D019923B9F0809396
:10112000E9008FEF9091E800815095FD06C095E1B0
:101130009A95F1F700008111F5CF8091E80085FFC5
:101140002CC040E050E060E170E017C081E0809387
:10115000E9008FEF9091E800815095FD06C095ED74
:101160009A95F1F700008111F5CF8091E80085FF95
:1011700014C040E050E068E070E0CE010E945F0AD9
:101180008091E8008E778093E80080E1FE01A2E57F
:10119000B1E001900D928A95E1F7DF91CF9108952A
:1011A0008091E301811109C00E94F00B0E944D0C57
:1011B0008091E20084608093E20008951092E30140
:1011C000089508950C949E210E94FE1A0E94A42165
:1011D0000E94F80E0C94EE0742E061EC81E00E9460
:1011E000690B42E061EC82E00E94690B42E061EC35
:1011F00083E00E94690B42E161EC84E00C94690B8E
:101200008091E601833009F455C030F4813071F0EB
:10121000823009F48EC008958A3009F47AC08B3088
:1012200009F460C0893009F09CC020C08091E501BC
:10123000813A09F096C08091E800877F8093E800AA
:101240008091E9019091EA01892B21F460E182E526
:1012500091E003C060E080E090E070E00E94AA0AA4
:101260008091E8008B778093E80008958091E501F4
:10127000813209F076C08091E9019091EA010097EE
:1012800019F0039709F06DC08091E800877F809383
:10129000E8008091E80082FD05C08091E4018111A1
:1012A000F8CF5FC08091F100809362018091E800E7
:1012B0008B7753C08091E501813A09F052C080914B
:1012C000E9019091EA01892B09F04BC08091E80077
:1012D000877F8093E8008091E80080FFFCCF8091B9
:1012E0000C0136C08091E5018132D9F58091E90188
:1012F0009091EA01892BA9F58091E800877F80937E
:10130000E8000E949E0B8091E70180930C010C94F1
:1013100061148091E501813221F58091E800877F99
:101320008093E8000E949E0B8091E8018093630106
:1013300008958091E501813AA1F48091E800877FCA
:101340008093E8008091E80080FFFCCF80916301EA
:101350008093F1008091E8008E778093E8000C94F0
:101360009E0B089584B7877F84BF0FB6F894A89525
:1013700080916000886180936000109260000FBED1
:1013800090E080E80FB6F89480936100909361003C
:101390000FBE0E94470F0E94F00B0E944D0C8091DF
:1013A000E20084608093E20078940E94D80E0E944C
:1013B000490F82E091E00E94F30E0E948C218091FF
:1013C000E401853069F40E94C01A8091E20188230B
:1013D000B1F30E94EA1A882391F30E94490AEFCFE1
:1013E0000E944F0FECCF292F332723303105C9F04E
:1013F00060F42130310581F02230310509F041C01F
:101400008DE690E020E634E040C021323105E1F085
:101410002232310531F135C082E190E02DEC34E02B
:1014200034C099278130910549F028F0029749F599
:10143000ECE2F4E005C0ECE5F4E002C0E4E4F4E042
:10144000849190E09F0121C06430D8F4E62FF0E051
:10145000EE0FFF1FEE5DFE4F2081318189E090E0AD
:1014600014C0643070F470E0FB01EE0FFF1FE65E05
:10147000FE4F20813181FB01EA5EFE4F808190E0CA
:1014800004C080E090E020E030E0FA013183208366
:10149000089580E189BD82E189BD09B400FEFDCFD8
:1014A0008091D8008F7D8093D8008091E000826089
:1014B0008093E0008091E00081FDFCCF0895CF9201
:1014C000DF92EF92FF920F931F93CF93DF93EC0184
:1014D0008B016A010E94BD0B811133C0C114D1047C
:1014E00039F0F60180819181081B190BC80FD91FB3
:1014F000E12CF12C0115110519F18091E80085FD11
:1015000016C08091E8008E778093E800C114D10462
:1015100049F0F60180819181E80EF91EF182E082A6
:1015200085E00FC00E94BD0B882321F30AC089917A
:101530008093F10001501109FFEFEF1AFF0ADACF93
:1015400080E0DF91CF911F910F91FF90EF90DF909E
:10155000CF9008952091EB013091EC0126173707C9
:1015600048F06115710539F42091E8002E77209339
:10157000E80001C0B901FC0120E06115710579F1B5
:101580008091E4018823F1F18530F1F18091E80048
:1015900083FD3CC08091E80082FD2EC08091E80070
:1015A00080FFEBCF2091F3008091F20090E0922B2E
:1015B0006115710551F08830910538F4219120931F
:1015C000F100615071090196F3CF21E0089709F00D
:1015D00020E08091E8008E778093E800CECF211143
:1015E000CFCF0AC08091E401882361F0853061F09B
:1015F0008091E80083FD0AC08091E80082FFF2CF6D
:1016000080E0089582E0089583E0089581E00895E0
:101610002091EB013091EC012617370748F0611556
:10162000710539F42091E8002E772093E80001C07D
:10163000B901FC0120E06115710591F18091E4018F
:10164000882309F440C0853009F43FC08091E80048
:1016500083FD3DC08091E80082FD2FC08091E800AD
:1016600080FFE9CF2091F3008091F20090E0922B6F
:101670006115710559F08830910540F4249120934B
:10168000F1003196615071090196F2CF21E008977F
:1016900009F020E08091E8008E778093E800CBCFBE
:1016A0002111CCCF0AC08091E401882361F08530FC
:1016B00061F08091E80083FD0AC08091E80082FF1C
:1016C000F2CF80E0089582E0089583E0089581E0FC
:1016D0000895982F973068F59093E900981739F09E
:1016E0007091EC002091ED005091F00003C0242F88
:1016F000762F50E021FD02C09F5FECCF3091EB00D0
:101700003E7F3093EB003091ED003D7F3093ED0054
:101710003091EB0031603093EB007093EC0020933C
:10172000ED005093F0002091EE0027FDE5CF80E022
:1017300008958F708093E90081E008958091E5011C
:1017400087FF11C08091E80082FD05C08091E4010F
:101750008111F8CF11C08091E8008B770BC0809188
:10176000E401882349F08091E80080FFF8CF809160
:10177000E8008E778093E80008952091E40030918E
:10178000E50095E64091EC00842F817040FF23C076
:101790008091E80080FD1DC08091E401882399F0CC
:1017A000853099F08091EB0085FD11C04091E400F7
:1017B0005091E5002417350729F3915011F09A0153
:1017C000E1CF84E0089582E0089583E0089581E008
:1017D000089580E008954091E80042FFDDCF08952C
:1017E0000E945E0C0E94660CE0EEF0E08081816059
:1017F0008083E8EDF0E080818F77808319BCA7EDCE
:10180000B0E08C918E7F8C9380818F7E808310924C
:10181000E30108950F931F93CF93DF930E945E0C13
:101820000E94660CC8EDD0E088818F77888388811C
:101830008068888388818F7D888319BC1092E40139
:101840001092E0011092E2011092E10100EE10E02E
:10185000F80180818B7F808388818160888342E06A
:1018600060E080E00E94690BE1EEF0E080818E7F15
:101870008083E2EEF0E080818160808380818860F7
:101880008083F80180818E7F808388818061888356
:10189000DF91CF911F910F910895E8EDF0E08081E5
:1018A0008F7E8083E7EDF0E080818160808384E03B
:1018B00082BF81E08093E3010C940A0CE8EDF0E034
:1018C00080818E7F80831092E20008951092DA006A
:1018D0001092E10008951F920F920FB60F921124FB
:1018E0002F933F934F935F936F937F938F939F9328
:1018F000AF93BF93EF93FF938091E10082FF0BC002
:101900008091E20082FF07C08091E1008B7F80938D
:10191000E1000E94D70E8091DA0080FF1FC0809105
:10192000D80080FF1BC08091DA008E7F8093DA00A0
:101930008091D90080FF0DC080E189BD82E189BD21
:1019400009B400FEFDCF81E08093E4010E94D0083D
:1019500005C019BC1092E4010E94DE088091E100EC
:1019600080FF19C08091E20080FF15C08091E200E5
:101970008E7F8093E2008091E20080618093E2009C
:101980008091D80080628093D80019BC85E0809354
:10199000E4010E94E2088091E10084FF30C0809160
:1019A000E20084FF2CC080E189BD82E189BD09B4D9
:1019B00000FEFDCF8091D8008F7D8093D80080916C
:1019C000E1008F7E8093E1008091E2008F7E809322
:1019D000E2008091E20081608093E2008091E0016A
:1019E000882311F084E007C08091E30087FD02C0E6
:1019F00081E001C083E08093E4010E94E4088091CB
:101A0000E10083FF29C08091E20083FF25C080911F
:101A1000E100877F8093E10082E08093E4011092EF
:101A2000E0018091E1008E7F8093E1008091E200EF
:101A30008E7F8093E2008091E20080618093E200DB
:101A400042E060E080E00E94690B8091F0008860D5
:101A50008093F0000E94E108FF91EF91BF91AF9158
:101A60009F918F917F916F915F914F913F912F91B6
:101A70000F900FBE0F901F9018951F920F920FB6E8
:101A80000F9211242F933F934F935F936F937F9304
:101A90008F939F93AF93BF93CF93DF93EF93FF9376
:101AA000C091E900CF708091EC00D82FD17080FDFB
:101AB000D0E81092E9008091F000877F8093F000D9
:101AC00078940E94810D1092E9008091F000886066
:101AD0008093F000CD2BCF70C093E900FF91EF9180
:101AE000DF91CF91BF91AF919F918F917F916F9136
:101AF0005F914F913F912F910F900FBE0F901F90CC
:101B000018951F93CF93DF93CDB7DEB7AA970FB683
:101B1000F894DEBF0FBECDBFE5EEF1E08091F1009D
:101B2000819321E0ED3EF207C9F70E940009809100
:101B3000E80083FF24C18091E5019091E601492FDF
:101B400050E04A30510508F01AC1FA01EA5AFF4F35
:101B50000C943523803881F0823809F010C18091CF
:101B6000E9018F708093E9008091EB0085FB882765
:101B700080F91092E90006C08091E1019091E201A4
:101B8000911182609091E800977F9093E800809394
:101B9000F1001092F100C8C0282F2D7F09F0EFC08E
:101BA000882319F0823061F0EAC08091E70181302A
:101BB00009F0E5C0933009F080E08093E2012BC08A
:101BC0008091E701811127C08091E9018F7009F4AC
:101BD000D6C08093E9002091EB0020FF1CC0933019
:101BE00021F48091EB00806214C09091EB00906131
:101BF0009093EB0021E030E0A90102C0440F551F93
:101C00008A95E2F74093EA001092EA008091EB0097
:101C100088608093EB001092E9008091E800877F54
:101C200086C08111ACC01091E7011F778091E3005D
:101C30008078812B8093E3008091E800877F8093F8
:101C4000E8000E949E0B8091E80080FFFCCF80910D
:101C5000E30080688093E300111102C082E001C0BC
:101C600083E08093E4018BC08058823008F087C005
:101C70008091E7019091E8018C3D53E0950779F55B
:101C800083E08A838AE289834FB7F894DE01139652
:101C900020E03EE051E2E32FF0E050935700E49162
:101CA00020FF03C0E295EF703F5FEF708E2F90E052
:101CB000EA3010F0C79601C0C0968D939D932F5FB8
:101CC000243149F74FBF8091E800877F8093E80077
:101CD0006AE270E0CE0101960E94AA0A14C0AE0129
:101CE0004F5F5F4F6091E9010E94F309BC01892BAE
:101CF00009F445C09091E800977F9093E8008981AE
:101D00009A810E94080B8091E8008B778093E8000D
:101D100036C08038A1F58091E800877F8093E80085
:101D20008091E0018093F1008091E8008E778093AC
:101D3000E8000E949E0B23C0811121C08091E70121
:101D40009091E80199270297D4F48091E800877F69
:101D50008093E8008091E7018093E0010E949E0B50
:101D60008091E001811106C08091E30087FD02C0EF
:101D700081E001C084E08093E4010E94EC0880913E
:101D8000E80083FF0AC08091E800877F8093E80025
:101D90008091EB0080628093EB00AA960FB6F894D6
:101DA000DEBF0FBECDBFDF91CF911F910895089583
:101DB000CF938091E4018823A1F0C091E900CF7016
:101DC0009091EC00892F817090FD80E8C82B1092D3
:101DD000E9008091E80083FD0E94810DCF70C093DF
:101DE000E900CF9108959093690180936801089567
:101DF000E0916801F0916901309721F00190F08144
:101E0000E02D099480E00895E0916801F091690166
:101E1000309721F00280F381E02D09940895E0913C
:101E20006801F0916901309721F00480F581E02D7F
:101E300009940895209166013091670128173907A8
:101E400071F09093670180936601E0916801F091D1
:101E50006901309721F00680F781E02D09940895FB
:101E600020916401309165012817390771F0909332
:101E7000650180936401E0916801F09169013097F8
:101E800021F00084F185E02D0994089508950C94C3
:101E9000460F0E94041B0E94B6040C94CA1BCF92EA
:101EA000DF92EF92FF920F931F93CF93DF93CDB703
:101EB000DEB72B970FB6F894DEBF0FBECDBF0E94E2
:101EC000CE048BE6C82E81E0D82E00E010E0E02E94
:101ED000802F0E94C405F60141916F01F82EF4266F
:101EE000B1F40F5F1F4F0E30110589F78FEF898313
:101EF0008A831B820E940D1B8160782F9D838C83B7
:101F000049815A816B818D810E94F20F40C090916E
:101F1000CC0191FF04C08B870E94CA058B8520E00D
:101F200030E04F2D50E0922FBA01022E02C075957D
:101F300067950A94E2F760FF24C02E83EF8221E0C8
:101F400030E0690102C0CC0CDD1C9A95E2F790E00C
:101F50008C219D21892B09F420E028870E940D1BEC
:101F60008160782F9A8789874E815F8168858A850D
:101F70000E94F20FF801E559FE4F8081C826C08209
:101F800006C02F5F3F4F2630310569F6AACF0E9469
:101F9000B11E0E94F80E90916A018917A1F00E946B
:101FA000F80E80936A012B960FB6F894DEBF0FBE31
:101FB000CDBFDF91CF911F910F91FF90EF90DF90F8
:101FC000CF900C94EE072B960FB6F894DEBF0FBEA1
:101FD000CDBFDF91CF911F910F91FF90EF90DF90D8
:101FE000CF900895CF93DF93CDB7DEB72B970FB681
:101FF000F894DEBF0FBECDBF4F83588769877A87BD
:102000008B87DE01119686E0FD0111928A95E9F732
:1020100085E0FE01379601900D928A95E1F749819E
:102020005A816B817C818D819E810E94F5162B9651
:102030000FB6F894DEBF0FBECDBFDF91CF910895EC
:10204000CF93C82F882309F4C1C0823859F40E9465
:10205000F80E81FDBBC089E30E9492190E944A1AC2
:1020600089E30CC0833879F40E94F80E80FDAEC07D
:1020700083E50E9492190E944A1A83E50E94D119B1
:10208000CF910C944A1A843859F40E94F80E82FDBC
:102090009DC087E40E9492190E944A1A87E4EECFFD
:1020A0008CEF8C0F813A48F48C2F0E94F120811123
:1020B0008DC08C2F0E949219E3CF80E28C0F883064
:1020C00048F4C77081E001C0880FCA95EAF70E9402
:1020D000131AD6CF8BE58C0F833078F4C53A29F0EC
:1020E000C63A31F083E890E005C081E890E002C094
:1020F00082E890E0CF910C941A0F88E58C0F833121
:1021000008F064C0C83A39F1C93A41F1CA3A49F114
:10211000CB3A51F1CC3A59F1CD3A61F1C03B69F17A
:10212000CE3A71F1CF3A79F1C13B81F1C23B89F1ED
:10213000C33B91F1C43B99F1C53BA1F1C63BA9F169
:10214000C73BB1F1C83BB9F1C93BC1F1CA3BC9F1C9
:1021500080E090E038C082EE90E035C089EE90E0FB
:1021600032C08AEE90E02FC085EB90E02CC086EB69
:1021700090E029C087EB90E026C08CEC90E023C073
:102180008DEC90E020C083E891E01DC08AE891E0EA
:102190001AC082E991E017C084E991E014C081E29D
:1021A00092E011C083E292E00EC084E292E00BC0A4
:1021B00085E292E008C086E292E005C087E292E004
:1021C00002C08AE292E0CF910C94300FCF91089533
:1021D000882309F44BC0823859F40E94F80E81FF1D
:1021E00045C089E30E9492190E944A1A89E30CC0F3
:1021F000833871F40E94F80E80FF38C083E50E9496
:1022000092190E944A1A83E50E94D1190C944A1A25
:10221000843859F40E94F80E82FF28C087E40E9497
:1022200092190E944A1A87E4EFCF9CEF980F913AD7
:1022300058F390E2980F983050F4877091E001C005
:10224000990F8A95EAF7892F0E94191ADFCF9BE52B
:10225000980F933020F480E090E00C941A0F885A85
:10226000833120F480E090E00C94300F08958823AF
:1022700021F00E94131A0C944A1A0895882321F021
:102280000E94191A0C944A1A0895BF92CF92DF92B5
:10229000EF92FF920F931F93CF93DF9300D000D064
:1022A00000D0CDB7DEB77C0185E0F701DE011196E5
:1022B00001900D928A95E1F7F70183819481892B32
:1022C00009F4DDC2908181818F3F19F49F3F09F4A9
:1022D000D6C2F7010281258122952F7099838A83C6
:1022E00089819A812E830E945119182FB92E0E943C
:1022F00050190E941718EB2DE295EF704E2F50E009
:10230000FA01E05AFF4F2E810C9435238B2D807FEC
:102310009B2D9F70F92E882319F0F29480EFF822FC
:10232000002349F0FF2009F457C28F2D0E94231A81
:102330000E944A1A51C2812F0E94E810FF2009F41E
:102340009EC28F2D0E94291A26960FB6F894DEBFE2
:102350000FBECDBFDF91CF911F910F91FF90EF90F6
:10236000DF90CF90BF900C944A1A3B2D307F8B2D7D
:102370008F70303211F08295807F112319F0113067
:1023800021F12CC00023B9F0222309F490C121309F
:1023900009F08DC126960FB6F894DEBF0FBECDBFF3
:1023A000DF91CF911F910F91FF90EF90DF90CF9031
:1023B000BF900C94331A222319F0213009F45FC224
:1023C0008E830E94361A8E8186C1002321F022302E
:1023D00008F055C26CC1211152C27DC1002321F009
:1023E000222309F464C1F8C1222309F474C109C28B
:1023F0008B2D86958695837019F08130D1F03FC280
:10240000002321F0812F9B2D937002C080E090E08B
:1024100026960FB6F894DEBF0FBECDBFDF91CF91E9
:102420001F910F91FF90EF90DF90CF90BF900C9491
:102430001A0F002321F0812F9B2D937002C080E0A2
:1024400090E026960FB6F894DEBF0FBECDBFDF91A9
:10245000CF911F910F91FF90EF90DF90CF90BF90A1
:102460000C94300F812F002319F00E94B91D02C077
:102470000E94211E26960FB6F894DEBF0FBECDBF78
:10248000DF91CF911F910F91FF90EF90DF90CF9050
:10249000BF900C94A61E8B2D837009F075C001119E
:1024A000EEC1812F829586958770880F880F912FB6
:1024B0009F70C92ED12CE12CF12C082E04C0CC0C1D
:1024C000DD1CEE1CFF1C0A94D2F714FF12C00FE0B3
:1024D00010E020E030E004C0000F111F221F331F66
:1024E0008A95D2F7C901B80160957095809590954D
:1024F00003C060E070E0CB014B2D469546954370DC
:102500004230C1F060F56C297D298E299F29413028
:1025100051F126960FB6F894DEBF0FBECDBFDF9106
:10252000CF911F910F91FF90EF90DF90CF90BF90D0
:102530000C943E186C297D298E299F2926960FB66A
:10254000F894DEBF0FBECDBFDF91CF911F910F91E9
:10255000FF90EF90DF90CF90BF900C945A180E949C
:102560003E18C701B60126960FB6F894DEBF0FBE1F
:10257000CDBFDF91CF911F910F91FF90EF90DF9032
:10258000CF90BF900C942218002319F08B2D8170EE
:1025900001C08695882309F472C1812F82958695A2
:1025A0008770880F880F912F9F70C92ED12CE12C36
:1025B000F12C082E04C0CC0CDD1CEE1CFF1C0A9470
:1025C000D2F714FF12C00FE010E020E030E004C0AA
:1025D000000F111F221F331F8A95D2F7C901B801BE
:1025E000609570958095909503C060E070E0CB0198
:1025F0004B2D4695469543704230C1F060F56C29ED
:102600007D298E299F29413051F126960FB6F894E5
:10261000DEBF0FBECDBFDF91CF911F910F91FF9015
:10262000EF90DF90CF90BF900C9418196C297D2902
:102630008E299F2926960FB6F894DEBF0FBECDBF18
:10264000DF91CF911F910F91FF90EF90DF90CF908E
:10265000BF900C9434190E941819C701B601269630
:102660000FB6F894DEBF0FBECDBFDF91CF911F91A3
:102670000F91FF90EF90DF90CF90BF900C94FC18DB
:10268000103FD1F118F4103E50F4A1C0123F09F4EC
:1026900063C008F44CC0133F09F473C098C01F70A6
:1026A0008B2D8F710023A1F00E949518812F269603
:1026B0000FB6F894DEBF0FBECDBFDF91CF911F9153
:1026C0000F91FF90EF90DF90CF90BF900C94371157
:1026D0000E94B618812F26960FB6F894DEBF0FBE63
:1026E000CDBFDF91CF911F910F91FF90EF90DF90C1
:1026F000CF90BF900C943E110023A9F02111BFC0D0
:102700008B2D8F7126960FB6F894DEBF0FBECDBF0E
:10271000DF91CF911F910F91FF90EF90DF90CF90BD
:10272000BF900C94DB18223008F0A9C0E9CF002339
:10273000A9F08B2D8F7126960FB6F894DEBF0FBED1
:10274000CDBFDF91CF911F910F91FF90EF90DF9060
:10275000CF90BF900C949518002359F38B2D8F7157
:1027600026960FB6F894DEBF0FBECDBFDF91CF9196
:102770001F910F91FF90EF90DF90CF90BF900C943E
:10278000B618002399F08B2D8F7126960FB6F8940A
:10279000DEBF0FBECDBFDF91CF911F910F91FF9094
:1027A000EF90DF90CF90BF900C94801826960FB6D4
:1027B000F894DEBF0FBECDBFDF91CF911F910F9177
:1027C000FF90EF90DF90CF90BF900C94761800238D
:1027D000A9F0222309F4ADCF812F26960FB6F894E5
:1027E000DEBF0FBECDBFDF91CF911F910F91FF9044
:1027F000EF90DF90CF90BF900C942010222309F42B
:10280000ADCF812F26960FB6F894DEBF0FBECDBF99
:10281000DF91CF911F910F91FF90EF90DF90CF90BC
:10282000BF900C94E8104B2D4F70612FC7010E9490
:10283000560326960FB6F894DEBF0FBECDBFDF91CC
:10284000CF911F910F91FF90EF90DF90CF90BF90AD
:102850000C949A174B2D4F70612FC70126960FB617
:10286000F894DEBF0FBECDBFDF91CF911F910F91C6
:10287000FF90EF90DF90CF90BF900C948B06269640
:102880000FB6F894DEBF0FBECDBFDF91CF911F9181
:102890000F91FF90EF90DF90CF90BF9008950E942E
:1028A000301A0E94051A0E944A1A0E94561F0E945E
:1028B000A61E80E090E00E941A0F80E090E00C9449
:1028C000300F0E94201A0C944F140E945119292F86
:1028D00022952F702C3030F42A3048F422502230C8
:1028E00078F405C02C3041F02F3031F009C0803E23
:1028F00048F0803F29F406C093FB882780F90895AB
:1029000080E0089581E00895CF93DF9300D000D058
:102910001F92CDB7DEB70F900F900F900F900F90D2
:10292000DF91CF910895CF93DF9300D000D000D0F6
:10293000CDB7DEB726960FB6F894DEBF0FBECDBF7B
:10294000DF91CF9108951F93CF93DF93C0917901C9
:1029500016E080917A01C81799F0D0E01C9FF00131
:102960001D9FF00D1124E558FE4F40815181628179
:102970007381848195810E9493142196C770E9CF59
:10298000DF91CF911F9108954091AB015091AC011F
:102990006091AD017091AE018091AF019091B00155
:1029A0000C9493148091B00182958F7009F054C0FB
:1029B0008091AD01882309F44FC080917901A091E5
:1029C0007A014091AE015091AF016091AB017091DD
:1029D000AC01B6E08A1709F43FC090E041155105FB
:1029E000C1F17F3F11F46F3FA1F1B89FF001B99F92
:1029F000F00D1124E558FE4F218127132AC02081B4
:102A0000261327C02281211124C023813481241759
:102A1000350710F421503109241B350B283C3105B2
:102A2000C0F42091B0012F7020612093B00126E006
:102A3000289FF001299FF00D1124E058FE4F80815E
:102A40008F70806180838BEA91E00E9445110C9425
:102A5000A31401968770BECF0895CF92DF92EF92B4
:102A6000FF920F931F93CF93DF93CDB7DEB762979B
:102A70000FB6F894DEBF0FBECDBF8C0185E0F80124
:102A8000DE011D9601900D928A95E1F7D8014C91D7
:102A900011965C91119712966C918091AE01909174
:102AA000AF01009709F475C13091AB017091AC0191
:102AB0007F3F19F43F3F09F46CC1F801C380D48013
:102AC000E090AD01EE2009F4BEC02091B001C8161F
:102AD000D90628F0D601A81BB90BCD0104C08095FA
:102AE00090958C0D9D1DFF24F394883C910578F002
:102AF000F12C207F09F0C4C07C2DD98AC88A89892D
:102B00000E9484148BEA91E00E944511AFC0822F8D
:102B1000807F09F045C0571313C0431311C06111E2
:102B20000FC02F7020612093B0010E94C4148BEA63
:102B300091E00E9445118091B001F80185832EC07B
:102B4000CD2819F15F3F11F44F3FF9F0F62E6111D6
:102B50001CC08091790120917A0136E0821709F436
:102B60005BC090E0389FF001399FF00D1124E558CB
:102B7000FE4F7181571306C07081471303C07281E5
:102B8000711103C001968770E9CFF62E662309F410
:102B90001CC18091B00181608093B001F12C15C1FE
:102BA000571309C0431307C0611105C08091B001DC
:102BB000F8018583C8C04D875E878D859E856A8BA9
:102BC0000E9465146A898823D1F16623C1F120919E
:102BD000B001822F82958F7090E0029774F08091FF
:102BE000AB019091AC0198878F831986DB86CA86EA
:102BF0002C87CE0107960E94451186E0F801ABEACA
:102C0000B1E001900D928A95E1F70E94D2140E94E2
:102C1000C414FF24F394D9C04D875E878D859E85AB
:102C20000E945119292F22952F70223008F0C1C01F
:102C30009F7009F0BBC0805E883008F4C6C0C80130
:102C40000E944511E6CFC816D90608F453C0F60114
:102C5000E81BF90BCF01883C910508F450C0F12C1A
:102C60007C2DD98AC88A89890E948414EBEAF1E014
:102C700086E0DF011D928A95E9F70E94C414A5C081
:102C8000571314C0431312C0611110C08091B001DA
:102C9000F8018583C8010E94451186E0EBEAF1E066
:102CA000DF011D928A95E9F7FE2C8FC04D875E8764
:102CB0008D859E856A8B0E9465146A89882309F434
:102CC000BECF662309F4BBCF2091B001822F82953D
:102CD0008F7090E002970CF490CF8091AB019091AF
:102CE000AC019A8389831B82DD82CC822E83CE0144
:102CF000019681CF809590958C0D9D1DACCFF62EC1
:102D0000662309F49CCF571333C0431331C020917D
:102D1000B00120FD24C0822F82958F70482F50E093
:102D200041155105E1F0D80115962C9315974F30B8
:102D3000510549F08F5F982F9295907F822F8F7069
:102D4000892B15968C93C8010E94451186E0F801E5
:102D5000ABEAB1E001900D928A95E1F78ECF86E063
:102D6000F801ABEAB1E001900D928A95E1F72DC030
:102D70004D875E878D859E850E94651481113DCFAC
:102D80008091B00181608093B001C8010E9445111B
:102D90001CC0662309F453CF4D875E878D859E85C1
:102DA0000E946514882309F44ACF27CF811143CFAD
:102DB0000CC0243008F043CF9F7009F43CCFD801F9
:102DC00015969C91907F09F036CF8F2D62960FB6A5
:102DD000F894DEBF0FBECDBFDF91CF911F910F9151
:102DE000FF90EF90DF90CF9008951F93CF93DF93E4
:102DF000CDB7DEB72C970FB6F894DEBF0FBECDBFB0
:102E00004F83588769877A878B879C87CE0107967F
:102E10000E942D15882371F08A859B85892B09F4E2
:102E200041C088858F3F09F065C08F818F3F09F0D1
:102E300061C038C086E0FE013796DE011196019030
:102E40000D928A95E1F76A857B856115710551F1CF
:102E5000FF81E885EF3F11F4FF3F21F120917A01D6
:102E600030E0C9010196877099274091790150E0BF
:102E70008417950709F447C0F983EA837D836C833F
:102E800096E0929FD001939FB00D1124A558BE4F9C
:102E9000FE01319601900D929A95E1F780937A01A7
:102EA0000E94A31416E08091790190917A0189170C
:102EB000B9F1189FC001112485589E4F0E942D150D
:102EC000882371F1E09179011E9FF0011124E558EA
:102ED000FE4F4081518162817381848195810E947E
:102EE00093148091790190E00196877099278093DF
:102EF0007901D9CF4F81588569857A858B859C85E5
:102F00000E949314CFCF0E94611410927A01109204
:102F10007901EBEAF1E086E0DF011D928A95E9F79D
:102F20002C960FB6F894DEBF0FBECDBFDF91CF91C8
:102F30001F910895EF92FF920F931F93CF93DF930A
:102F40008C01892B09F46CC0F12CEE24E394E80188
:102F50002196F8018491843740F4843008F051C000
:102F6000813081F0823019F15BC0853709F444C0AB
:102F7000A8F19CE7980F903708F052C08F770E9415
:102F8000E81041C00E5F1F4FFE01849190E2980F40
:102F9000983050F48770FE2D01C0FF0F8A95EAF734
:102FA0008F2F0E94231A14C00E9420102DC00E5F84
:102FB0001F4FFE01849190E2980F983060F4877063
:102FC000FE2D01C0FF0F8A95EAF78F2F0E94291A64
:102FD0000E944A1A19C00E94E81016C00E5F1F4FC7
:102FE000FE01C491CC2381F08FE99FE00197F1F7B6
:102FF00000C00000C150F6CF0E5F1F4FFE01F490DD
:1030000003C00E9420108E018F2D882309F49FCFCA
:10301000EFE9FFE03197F1F700C000008150F5CFF4
:10302000DF91CF911F910F91FF90EF900895089538
:103030006093B5017093B6018093B7019093B80186
:103040000C944F140F931F930091B5011091B6018A
:103050002091B7013091B801DC01CB01802B912B7D
:10306000A22BB32B8093B5019093B601A093B70127
:10307000B093B8011F910F910C944F140F931F93AD
:103080000091B5011091B6012091B7013091B801BE
:10309000DC01CB0180239123A223B3238093B501CC
:1030A0009093B601A093B701B093B8011F910F910F
:1030B0000C944F140F931F930091B5011091B6011A
:1030C0002091B7013091B801DC01CB018027912715
:1030D000A227B3278093B5019093B601A093B701BF
:1030E000B093B8011F910F910C944F141092B1013D
:1030F0001092B2011092B3011092B4010C944F14CB
:1031000041E050E060E070E004C0440F551F661FCE
:10311000771F8A95D2F74093B1015093B201609323
:10312000B3017093B4010C944F1441E050E060E09F
:1031300070E004C0440F551F661F771F8A95D2F7B1
:103140008091B1019091B201A091B301B091B4010D
:10315000482B592B6A2B7B2B4093B1015093B20122
:103160006093B3017093B4010C944F1441E050E0AC
:1031700060E070E004C0440F551F661F771F8A95FA
:10318000D2F740955095609570958091B1019091DE
:10319000B201A091B301B091B401482359236A232D
:1031A0007B234093B1015093B2016093B3017093BC
:1031B000B4010C944F1441E050E060E070E004C0B2
:1031C000440F551F661F771F8A95D2F78091B10172
:1031D0009091B201A091B301B091B4014827592751
:1031E0006A277B274093B1015093B2016093B301EA
:1031F0007093B4010C944F140F931F930091B1017D
:103200001091B2012091B3013091B401DC01CB01E6
:10321000802B912BA22BB32B8093B1019093B20101
:10322000A093B301B093B4011F910F910C944F146C
:103230000F931F930091B1011091B2012091B3013E
:103240003091B401DC01CB0180239123A223B3236D
:103250008093B1019093B201A093B301B093B401F4
:103260001F910F910C944F140F931F930091B10174
:103270001091B2012091B3013091B401DC01CB0176
:1032800080279127A227B3278093B1019093B201A1
:10329000A093B301B093B4011F910F910C944F14FC
:1032A0000895CF92DF92EF92FF920F931F93CF93E7
:1032B000DF938C01C090B101D090B201E090B301D6
:1032C000F090B4018091B5019091B601A091B70141
:1032D000B091B801C82AD92AEA2AFB2ACFE1D0E066
:1032E000D701C6010C2E04C0B695A7959795879572
:1032F0000A94D2F780FF07C0B8018C2F0E94AF0656
:103300008130910531F4219758F7B80180E00E948F
:10331000AF06DF91CF911F910F91FF90EF90DF905B
:10332000CF90089590910C019923F1F090910D01A7
:103330009923D1F0982F9695969596959F3080F584
:10334000E0910E01F0910F01E90FF11D877021E06E
:1033500030E0A90102C0440F551F8A95E2F7CA0167
:103360009181892B8183089520910E0130910F0165
:10337000F90132969FEF40E05191851789F09F3F08
:1033800019F4511101C0942F4F5F4E30A9F79F3FA0
:1033900039F0F901E90FF11D97FDFA95828308953F
:1033A000089590910C019923F9F090910D019923C2
:1033B000D9F0982F9695969596959F3028F5E0919F
:1033C0000E01F0910F01E90FF11D877021E030E04F
:1033D000A90102C0440F551F8A95E2F7CA018095E2
:1033E000918189238183089520910E0130910F01ED
:1033F000F9013296205F3F4F9081891301C01082FE
:103400003196E217F307C1F7089581E090E0E0916B
:103410000E01F0910F01E80FF91F10820196803123
:103420009105A9F708959091CB01892B8093CB0149
:10343000089580959091CB0189238093CB010895C5
:103440001092CB0108959091CA01892B8093CA01F3
:10345000089580959091CA0189238093CA010895A7
:103460001092CA0108958093B90108951092B9018C
:10347000089580910E0190910F01FC0131969C01FD
:10348000205F3F4F80E0919191118F5FE217F3072A
:10349000D1F70895E0910E01F0910F018091CB01D9
:1034A0008083E0910E01F0910F0190818091CA011B
:1034B000892B80838091B901882361F0E0910E010E
:1034C000F0910F019081892B80830E94391A81111C
:1034D0001092B90180910E0190910F010C94040F8C
:1034E000CF92DF92EF92FF926C01EE24FF24C11481
:1034F000D104E104F10421F0C701B60120E101C0CB
:1035000020E0C72ED82EE92EFF24C114D104E104F7
:10351000F10419F0285FC701B6016B017C0154E08A
:10352000F694E794D794C7945A95D1F7C114D1046F
:10353000E104F10419F02C5FC701B6016B017C01B5
:1035400042E0F694E794D794C7944A95D1F7C11412
:10355000D104E104F10419F02E5FC701B601DC01CA
:10356000CB01B695A79597958795892B8A2B8B2BA1
:1035700009F02F5F822FFF90EF90DF90CF9008959A
:103580008091E401843011F120E488E190E00FB6ED
:10359000F894A895809360000FBE2093600083B7D5
:1035A000817F846083BF83B7816083BF789488956F
:1035B00083B78E7F83BF0FB6F894A8958091600083
:1035C000886180936000109260000FBE0895089596
:1035D0000C94E71ACF930E94E81A0E94CE040E942E
:1035E000E71AC0E08C2F0E94C405811104C0CF5F90
:1035F000CE30C1F701C081E0CF9108950E946114DF
:103600000E94F80E0C94EE0782E084BD93E095BD15
:103610009AEF97BD80936E0008952FB7F89480912C
:10362000CD019091CE01A091CF01B091D0012FBFDB
:103630000895CF92DF92EF92FF920F931F932FB7CF
:10364000F8944091CD015091CE016091CF017091DD
:10365000D0012FBF6A017B01EE24FF248C0120E002
:1036600030E0C016D106E206F30610F441505109CD
:103670009A01281B390BC9011F910F91FF90EF9000
:10368000DF90CF9008951F920F920FB60F921124E2
:103690008F939F93AF93BF938091CD019091CE0173
:1036A000A091CF01B091D0010196A11DB11D8093D1
:1036B000CD019093CE01A093CF01B093D001BF91E3
:1036C000AF919F918F910F900FBE0F901F90189503
:1036D0000E94F00BF8942FEF87EA91E6215080408A
:1036E0009040E1F700C0000087E090EBDC018093A0
:1036F000ED019093EE01A093EF01B093F0019CE0F7
:1037000088E10FB6F894A895809360000FBE90935F
:103710006000FFCFEF92FF920F931F93CF93DF9341
:10372000D82FC0E08C2F0E94C40500E010E0E82EE6
:10373000F12CC701002E02C0959587950A94E2F7F7
:1037400080FD06C00F5F1F4F0630110591F709C0BD
:10375000602F7C2F80E00E948C068D13F3CF81E0D8
:1037600004C0CF5FCE30F1F680E0DF91CF911F91A2
:103770000F91FF90EF900895CF93C82F8CE20E9495
:103780008A1B882321F08C2FCF910C948A1B80E018
:10379000CF910895CF930E94111D811102C00E9404
:1037A000F71CC5E6C15049F00E94CE048FE39CE9A6
:1037B0000197F1F700C00000F5CF89E20E94BC1B21
:1037C000811113C18AE20E94BC1B81110E94F71C67
:1037D00085E00E94BC1B81110E94681B0E941C1D79
:1037E0008093CC0187E00E94BC1B8823A9F18BE168
:1037F0000E94BC1B882351F08091CC0181FB2227C1
:1038000020F991E0922790FB81F90EC08EE00E9492
:10381000BC1B882361F08091CC0182FB222720F918
:1038200091E0922790FB82F98093CC0115C080E152
:103830000E94BC1B9091CC01882341F093FB22276E
:1038400020F981E0822780FB93F904C0892F8095BD
:1038500080FB90F99093CC018091CC010E94201DB7
:103860000E942E1D8093DE0180EE0E94BC1B8823E7
:1038700041F08091DE01982F909590FB80F9809324
:10388000DE0189E30E94BC1B882359F08091DE0190
:1038900081FB222720F991E0922790FB81F9809308
:1038A000DE0182EE0E94BC1B882359F08091DE016C
:1038B00082FB222720F991E0922790FB82F98093E6
:1038C000DE0186EE0E94BC1B882359F08091DE0148
:1038D00083FB222720F991E0922790FB83F98093C4
:1038E000DE0183EE0E94BC1B882359F08091DE012B
:1038F00084FB222720F991E0922790FB84F98093A2
:10390000DE0185E30E94BC1B882359F08091DE0113
:1039100085FB222720F991E0922790FB85F980937F
:10392000DE0181E30E94BC1B882359F08091DE01F7
:1039300086FB222720F991E0922790FB86F980935D
:10394000DE0181E10E94BC1B882359F08091DE01D9
:1039500087FB222720F991E0922790FB87F980933B
:10396000DE018091DE010E94321D8091DE0187FB25
:10397000882780F980930D0187E20E94BC1BC82F25
:103980008EE10E94BC1B8111C2608FE10E94BC1BB2
:103990008111C46080E20E94BC1B8111C86081E279
:1039A0000E94BC1B8111C06182E20E94BC1B81117C
:1039B000C06283E20E94BC1B8111C06484E20E9449
:1039C000BC1B882311F0C06802C0CC2329F08C2FC7
:1039D0000E94291D6C2F03C00E94251D682F70E0D6
:1039E00080E090E0CF910C941818CF9108956DEE7F
:1039F0007EEF80E090E00E946B2360E082E090E048
:103A00000E945D2360E083E090E00E945D2360E01F
:103A100084E090E00E945D2360E085E090E00C94FB
:103A20005D2380E090E00E94572321E08D3E9E4F71
:103A300009F020E0822F089582E090E00C944F235B
:103A4000682F82E090E00C945D2383E090E00C947A
:103A50004F23682F83E090E00C945D2384E090E096
:103A60000C944F23682F84E090E00C945D238091A8
:103A7000D30180FF0BC06091130185E0689FB00106
:103A8000112475956795759567952BC081FF09C0C1
:103A90006091130185E0689FB001112475956795C9
:103AA00020C082FF07C06091130185E0689FB001CC
:103AB000112417C09091D4019923D1F06091120183
:103AC000961788F72091130185E0289F9001112413
:103AD000929FA001939F500D112470E0CA010E9493
:103AE00021236038710540F46115710519F406C091
:103AF00065E070E0862F08958FE7089581E00895CE
:103B00008091D30180FF08C06091110170E075952C
:103B100067957595679521C081FF06C06091110179
:103B200070E07595679519C082FF04C0609111011E
:103B300070E010C09091D401992399F06091100128
:103B40009617A0F780911101899FC001112470E0A0
:103B50000E9421236038710540F46115710519F444
:103B600006C061E070E0862F08958FE7089581E038
:103B70000895803F21F40E94371D819504C0813F44
:103B800029F40E94371D8093D7010895823F21F4C4
:103B90000E94371D819504C0833F29F40E94371D80
:103BA0008093D6010895893F19F40E94801D05C0B5
:103BB0008A3F31F40E94801D81958093D801089539
:103BC0008B3F21F40E94801D819504C08C3F29F415
:103BD0000E94801D8093D9010895843F21F4809133
:103BE000D501816017C0853F21F48091D5018260A5
:103BF00011C0863F21F48091D50184600BC0873FBE
:103C000021F48091D501886005C0883F31F480910E
:103C1000D50180618093D50108958D3F21F4809175
:103C2000D30181600BC08E3F21F48091D30182606B
:103C300005C08F3F29F48091D30184608093D30124
:103C40000895803F39F48091D70187FF6CC01092AE
:103C5000D70169C0813F29F48091D7011816BCF3C0
:103C600062C09091D601823F29F497FF5CC0109208
:103C7000D60159C0833F19F41916CCF354C0893FBB
:103C800041F48091D80118160CF04DC01092D80163
:103C90004AC08A3F29F48091D80187FF44C0F6CFFB
:103CA0008B3F39F48091D90187FF3DC01092D90133
:103CB0003AC08C3F29F48091D9011816BCF333C067
:103CC000843F21F48091D5018E7F17C0853F21F478
:103CD0008091D5018D7F11C0863F21F48091D5015F
:103CE0008B7F0BC0873F21F48091D501877F05C072
:103CF000883F31F48091D5018F7E8093D50113C028
:103D00008D3F21F48091D3018E7F0BC08E3F21F433
:103D10008091D3018D7F05C08F3F29F48091D3011D
:103D20008B7F8093D3018091D60181110EC0809149
:103D3000D70181110AC08091D801811106C08091FC
:103D4000D901811102C01092D401089585ED91E04E
:103D50000E940F0F0E940D1B9093D2018093D101FE
:103D600008951F93CF93DF938091D1019091D20159
:103D70000E94191BAC019091D401992321F020914C
:103D8000140130E006C0209115018AE0289F9001BF
:103D900011244217530708F485C08091D601C091C1
:103DA000D701D091D8011091D901811107C0C1115B
:103DB00075C0D11173C0111171C074C09F3F19F04B
:103DC0009F5F9093D401181624F40E94371D8093AE
:103DD000D6018091D60187FF05C00E94371D8195CD
:103DE0008093D6011C1624F40E94371D8093D701BE
:103DF0008091D70187FF05C00E94371D8195809370
:103E0000D7016091D601662331F1C091D701CC234F
:103E100011F1062E000C770B880B990B0E942822BB
:103E200023E333E343E35FE30E948C220E94F0210B
:103E30006093D6016C2FCC0F770B880B990B0E94E7
:103E4000282223E333E343E35FE30E948C220E94B2
:103E5000F0216093D7011D1624F40E94801D8093E9
:103E6000D8018091D80187FF05C00E94801D8195EF
:103E70008093D801111624F40E94801D8093D901EB
:103E80008091D90187FF05C00E94801D8195809394
:103E9000D901DF91CF911F910C94A61E9F3F09F08D
:103EA0008FCFA0CFDF91CF911F910895E5EDF1E085
:103EB00085E0DF011D928A95E9F71092D4011092F6
:103EC000D3010895833081F128F4813059F0823094
:103ED000D1F00895853009F449C0B8F1863009F46D
:103EE00056C0089580911501262F30E0280F311D0E
:103EF0002F3F310524F4680F6093150108958FEF6B
:103F000080931501089580911401262F30E0280F29
:103F1000311D2F3F310524F4680F6093140108957B
:103F20008FEF80931401089580911301262F30E0C4
:103F3000280F311D2F3F310524F4680F60931301C2
:103F400008958FEF80931301089580911201262F19
:103F500030E0280F311D2F3F310524F4680F6093A6
:103F6000120108958FEF809312010895809111013D
:103F7000262F30E0280F311D2F3F310524F4680F24
:103F80006093110108958FEF80931101089580913E
:103F90001001262F30E0280F311D2F3F310524F46A
:103FA000680F6093100108958FEF809310010895BA
:103FB000833011F128F4813049F0823091F0089576
:103FC000853081F120F18630C1F10895809115018D
:103FD000681720F4861B809315010895109215012F
:103FE000089580911401681720F4861B80931401B2
:103FF000089510921401089580911301681720F418
:10400000861B8093130108951092130108958091E7
:104010001201681720F4861B8093120108951092F4
:104020001201089580911101681720F4861B809376
:1040300011010895109211010895809110016817DF
:1040400020F4861B809310010895109210010895AA
:104050000F931F938D3109F46BC008F03FC08E3071
:1040600009F47DC0C0F4873009F46EC068F486306E
:1040700009F0AFC08091CC01817F8E7F8093CC010D
:1040800081E08093DB01A6C0883009F458C08B30F2
:1040900009F49BC09EC0863109F497C078F4803142
:1040A00009F470C0813109F094C00E9461149091AC
:1040B0000D0181E0892780930D0187C0893109F4C2
:1040C00084C08B3109F085C08091CC0181FB22270F
:1040D00020F991E0922790FB81F94AC0853309F4D9
:1040E0005BC048F4873209F457C008F45AC08932DB
:1040F00009F452C06EC0833438F48A3308F067C0C4
:10410000883309F462C065C0833409F445C088343B
:1041100009F05FC00E9461140FEF13ED20E301501E
:1041200010402040E1F700C000000E94681B4DC015
:104130000E94AA210E94F80E0E94EE0746C00E942B
:104140001C1D0E942E1D41C09091CC01892F8170B1
:1041500090FF12C0917F9E7F9093CC013BC08091D5
:10416000CC0182FB222720F991E0922790FB82F973
:104170008093CC01992349F18091CC018160809397
:10418000CC0123C08091CC0183FB222720F991E050
:10419000922790FB83F9ECCF61E070E080E090E043
:1041A00010C08D5141E050E060E070E08A019B0159
:1041B00004C0000F111F221F331F8A95D2F7C901B7
:1041C000B8010E9418180E94611481E003C089534D
:1041D000E9CF80E01F910F91089580E008950C943D
:1041E000ED20CF93C82F8091DB01813079F018F05A
:1041F0008230E9F187C0E0910E01F0910F018081DA
:10420000813169F0823209F07FC009C0E0910E016E
:10421000F0910F018081813111F0823261F48C2F95
:104220000E94EF20811104C08C2F0E9428201DC005
:1042300081E090E01AC08C2F0E94ED20811114C003
:10424000C43179F048F4CB3079F0C03109F060C066
:1042500082E08093DB0108C0C93219F0C83321F035
:1042600057C01092DB0154C081E0817053C0C93245
:1042700089F118F5C43171F1A8F4C73009F046C0CE
:104280008AE08093150194E19093140193E0909358
:1042900013018093120188E08093110188E28093DA
:1042A000100134C0CE51C63088F5EC2FF0E0E65D49
:1042B000FE4F80818093DA0129C0CE34E9F020F4EA
:1042C000CB3421F56AE013C0C13579F0C235F1F481
:1042D00061E00DC08091DA01882319F01092DA01B3
:1042E00015C081E08093DB0115C061E006C08091BC
:1042F000DA010E94621F0AC06AE08091DA010E941E
:10430000D81F04C01092DB0180E004C081E002C02D
:1043100080E0ABCFCF910895E1E8F0E08081886044
:1043200080838081816080838FB7F89493E090933D
:10433000890090ED909388008FBF0895EFE6F0E03C
:104340008081826080830895EFE6F0E080818D7F38
:1043500080830895EFE6F0E0908182E089278083F2
:1043600008951F920F920FB60F9211242F933F932F
:104370004F935F936F937F938F939F93AF93BF936D
:10438000EF93FF938091DC019091DD010196909372
:10439000DD018093DC01811103C082E00E94EE0701
:1043A000E091DD01E695E695F0E0E652FA4FE49102
:1043B0008091DC018E1303C080E00E94EE07FF9124
:1043C000EF91BF91AF919F918F917F916F915F918D
:1043D0004F913F912F910F900FBE0F901F90189506
:1043E0000E94F7216894B1110C94862208950E94CE
:1043F0006B2288F09F5798F0B92F9927B751B0F0EA
:10440000E1F0660F771F881F991F1AF0BA95C9F758
:1044100014C0B13091F00E948522B1E008950C944F
:104420008522672F782F8827B85F39F0B93FCCF302
:10443000869577956795B395D9F73EF490958095D5
:10444000709561957F4F8F4F9F4F0895E89409C0F5
:1044500097FB3EF490958095709561957F4F8F4FB7
:104460009F4F9923A9F0F92F96E9BB279395F695CD
:10447000879577956795B795F111F8CFFAF4BB0F4B
:1044800011F460FF1BC06F5F7F4F8F4F9F4F16C0AF
:10449000882311F096E911C0772321F09EE8872F39
:1044A000762F05C0662371F096E8862F70E060E0F5
:1044B0002AF09A95660F771F881FDAF7880F96956E
:1044C000879597F9089557FD9058440F551F59F057
:1044D0005F3F71F04795880F97FB991F61F09F3FF1
:1044E00079F087950895121613061406551FF2CF1A
:1044F0004695F1DF08C0161617061806991FF1CF6A
:1045000086957105610508940895E894BB27662790
:104510007727CB0197F908950E949F220C941023CE
:104520000E94022338F00E94092320F0952311F005
:104530000C94F9220C94FF2211240C9486220E94E0
:10454000632270F3959FC1F3950F50E0551F629F52
:10455000F001729FBB27F00DB11D639FAA27F00DDC
:10456000B11DAA1F649F6627B00DA11D661F829F03
:104570002227B00DA11D621F739FB00DA11D621FE8
:10458000839FA00D611D221F749F3327A00D611D05
:10459000231F849F600D211D822F762F6A2F1124E7
:1045A0009F5750409AF0F1F088234AF0EE0FFF1F1A
:1045B000BB1F661F771F881F91505040A9F79E3F71
:1045C000510580F00C94F9220C9486225F3FE4F3AD
:1045D000983ED4F3869577956795B795F795E795C7
:1045E0009F5FC1F7FE2B880F911D9695879597F9D0
:1045F000089597F99F6780E870E060E008959FEF65
:1046000080EC089500240A94161617061806090669
:10461000089500240A941216130614060506089538
:10462000092E0394000C11F4882352F0BB0F40F4C0
:10463000BF2B11F460FF04C06F5F7F4F8F4F9F4F00
:10464000089597FB072E16F4009407D077FD09D044
:104650000E943B2307FC05D03EF4909581959F4F27
:104660000895709561957F4F0895EE0FFF1F059097
:10467000F491E02D0994AA1BBB1B51E107C0AA1FAE
:10468000BB1FA617B70710F0A61BB70B881F991FF3
:104690005A95A9F780959095BC01CD010895F99997
:1046A000FECF92BD81BDF89A992780B50895A8E103
:1046B000B0E042E050E00C947223262FF999FECF2F
:1046C0001FBA92BD81BD20BD0FB6F894FA9AF99A2F
:1046D0000FBE019608950E945D23272F0C945E2340
:1046E000DC01CB01FC01F999FECF06C0F2BDE1BDB2
:1046F000F89A319600B40D9241505040B8F70895A1
:04470000F894FFCF5B
:104704002002EF077F085A082608F2070101BA01C0
:1047140028080A03140A3F4D36399B054E0518052F
:10472400DF0472048B04A404BD040102030405061F
:044734000708090069
:00000001FF
